:020000040000FA
:1000000083162B3085008113831207309900A501D8
:10001000851A56280030842000281E30A9000000D0
:10002000AA0B0F28A90B0F2800343C30A7000000B2
:10003000A60B1728A70B1728003400001F28A60BB3
:100040001D28A70B1D2800341D201D201D201D204C
:100050000034A400A300A3090310A30C0310230C75
:1000600023072408A100051505123628372838284B
:100070000000A10B35282408A10005110516402811
:10008000851E612843280000A10B3F28A30B3128BF
:100090000D200034A400A300A3093128A40060307F
:1000A000A3003128A400FF30A300312883169B0150
:1000B0001C141A088312A50000302506031D6628AB
:1000C000E82B2620A50AA50A2508842025088207F2
:1000D000952068281D216A2852216C2894216E28B9
:1000E000F621702851227228A3227428E82276284B
:1000F000302378286A237A28B3237C280000851EC1
:100100007F281D20A501E82B83169B019A001C1552
:1001100055309D00AA309D009C1483128C1F8E28A0
:100120008C1383161C1183120034973029208E30D3
:10013000292080304A204B304A205F304A205430FA
:1001400029205F3029205F304A2066304A206630FF
:100150004A20AC302920973029208E304A20543054
:100160004A2066304A205F302920663029207130CD
:100170004A2080304A2080304A20973029208E3013
:10018000292080304A205F302920543029204B30EC
:100190004A20543029205F30292071304A205430C1
:1001A00029204B30292047304A2015204B30292068
:1001B0006630292071304A2047304A204B304A208F
:1001C000543029205F304A201D205F304A205F30A4
:1001D00029204B304A205F304A2054304A20543086
:1001E000292054304A201D2054304A2054302920E0
:1001F00047304A2054304A204B304A204B30292087
:100200004B304A201D204B304A204B3029204030B3
:100210004A2047304A2047304A204730292047307B
:100220004A204B3029205430292080304A20663023
:100230004A205F304A20242000349730292097300C
:10024000292097304A20973029209730292097304D
:100250004A209730292080302920C0302920AC3016
:100260004A2097304A201D208E3029208E302920A8
:100270008E3029208E3029208E3029209730292059
:10028000973029209730292097302920AC30292019
:10029000AC30292097302920AC304A2080304A20C9
:1002A00024200034803029208030292080304E20C6
:1002B000AC304E201D206630292066302920663063
:1002C0004E2080304E201D2080302920663029208D
:1002D00054304A2054304E205F304E2066304E203D
:1002E00071304E201D2071304A2066304A205F3028
:1002F0004A205F30292066304E2071304E20663013
:100300004E2080304E201D2080304E2066304E2002
:1003100071304E20AC304E208E304E2071304E2049
:1003200080304E2024200034543029204B302920A6
:100330005F30292071302920152066302920803037
:10034000292015201520543029204B3029205F30DA
:1003500029207130292015206630292080304A203C
:10036000AC30292097304A20C0304A20E3304E205C
:100370001520CA304E20E3304E20F2304E2015209A
:10038000F5304E201520AC302920A03029209730A0
:1003900029205F3029201520973029205F3029201F
:1003A0001520973029205F304A2015205F30292002
:1003B0004B302920493029204B3029205F3029201B
:1003C000553029204B3029204B30292066302920F8
:1003D00054304A205F304A2015205F3029201520F4
:1003E000AC302920A030292024200034C0304A20FD
:1003F000C0304A2080304A2080304A2071304A2064
:1004000071304A2080304A201D208E304A208E30A4
:100410004A2097304A2097304A20AC304A20AC30EE
:100420004A20C0304A201D2080304A2080304A2097
:100430008E304A208E304A2097304A2097304A200A
:10044000AC304A201D2080304A2080304A208E3037
:100450004A208E304A2097304A2097304A20AC30CC
:100460004A201D20C0304A20C0304A2080304A2017
:1004700080304A2071304A2071304A2080304A2032
:100480001D208E304A208E304A2097304A209730E7
:100490004A20AC304A20AC304A20C0304A202420C8
:1004A0000034AC302920803029207130292066307A
:1004B0004A2066304A201D20663029206B302920D2
:1004C0006230292080304A2080304A201D20803030
:1004D000292071302920663029204B304A204B30AA
:1004E0004A201D204B302920543029205F302920FC
:1004F00066304A201D208030292071302920663046
:10050000292054304A204B304A201D204B302920CE
:10051000543029205F30292066304A2080304A201C
:100520001D20803029207130292066304A205F301C
:10053000292071304A2071302920663029208030EE
:100540004A2024200034C0304A20AC304A20973062
:100550004A20C0304A20C0304A20AC304A20973070
:100560004A20C0304A201D2097304A208E304A2031
:1005700080304E2097304A208E304A2080304E20E6
:100580001D208030292071302920803029208E3094
:10059000292097304A20C0304A20803029207130ED
:1005A0002920803029208E30292097304A20C030E1
:1005B0004A201D20C0304E20CC304E20C0304E206E
:1005C000C0304E20CC304E20C0304E20242000348D
:1005D00080302920663029205F30292054304A207D
:1005E0001D2080302920663029205F30292054309A
:1005F0004A201D2080302920663029205F302920A4
:1006000054304A2066304A2080304A2066304A20E2
:1006100071304A201D206630292066302920713033
:10062000292080304A208030292066304A205430EA
:10063000292054302920543029205F304A201D20A1
:100640004B304A204B30292054304A2066304A2013
:1006500071304A207130292080304A202420003413
:1006600097302920AC302920C0302920AC304E20D2
:100670009730292097302920973029201D20AB3032
:100680002920AC302920AC304E201D209730292065
:100690008030292080304E201D2092302920AC301F
:1006A0002920C0302920AC3029208E3029208E30DE
:1006B00029208E304E201D2097302920AC30292053
:1006C000AC30292097302920AC302920C0304E2072
:1006D00024200034803029209730292080304E207B
:1006E0001D20803029209730292080304E201D2069
:1006F00071302920803029208E3029209730292000
:10070000AC302920973029208E3029201D209730A9
:1007100029208E30292080304E201520C0304E20D8
:100720001520C0302920C0302920C0304E201D2087
:10073000C0302920AC302920973029208E30292044
:1007400080304E201D2080302920AC302920AC3054
:1007500029208E30292097302920AC302920C03024
:100760004E202420003480304A2080304A207130CE
:100770004A2080304A205F304A2066304A201D20BF
:1007800080304A2080304A2071304A2080304A2010
:1007900054304A205F304A201D2080304A2080306B
:1007A0004A20403052204B3052205F304A20663081
:1007B0004A2071304A201D20473052204B305220B1
:1007C0005F304A2054304A205F304A2024200034D1
:1007D000952095201D211D215221522194219421E3
:1007E000F621F62151225122A322A322E822E82257
:0E07F000302330236A236A23B323B323002867
:02400E00D43F9D
:024200000000BC
:00000001FF
